:0200000480007A
:100000006F008004732F2034930F80006308FF0378
:10001000930F90006304FF03930FB0006300FF038E
:10002000130F000063040F0067000F00732F2034CC
:1000300063540F006F00400093E19153171F0000BD
:1000400023223FFC6FF09FFF93000000130100008C
:10005000930100001302000093020000130300004C
:100060009303000013040000930400001305000034
:10007000930500001306000093060000130700001C
:100080009307000013080000930800001309000004
:1000900093090000130A0000930A0000130B0000EC
:1000A000930B0000130C0000930C0000130D0000D4
:1000B000930D0000130E0000930E0000130F0000BC
:1000C000930F0000732540F16310050097020000B4
:1000D000938202017390523073500018970200000F
:1000E00093824202739052309B021000939252030B
:1000F0009382F2FF7390023B9302F0017390023AF5
:100100007350403097020000938242017390523046
:10011000735020307350303093010000970200007C
:10012000938282EE73905230130510001315F5017F
:10013000635C05000F00F00F930110009308D005D9
:10014000130500007300000093020000638A0200A0
:1001500073905210B7B200009B82921073902230BD
:100160007350003037250000732005307350300085
:10017000970200009382420173901234732540F17C
:10018000730020301B05F01F13157501530505F092
:10019000531505E09303100093012000631C750EB6
:1001A0001B05F01713157501530505F0531505E0F0
:1001B0009303200093013000631E750C1B05101083
:1001C000131575011305F5FF530505F0531505E0EB
:1001D0009303400093014000631E750A1B05100045
:1001E0001315F501530505F0531505E09303800041
:1001F000930150006310750A13050000530505F0C4
:10020000531505E093030001930160006314750822
:10021000370580001B05F5FF530505F0531505E074
:100220009303000293017000631675063705803F43
:10023000530505F0531505E0930300049301800076
:10024000631A75043705807F530505F0531505E0E3
:100250009303000893019000631E75023705807FA9
:100260001B051500530505F0531505E09303001019
:100270009301A000631075023705C07F530505F098
:10028000531505E0930300209301B000631475003B
:10029000631030020F00F00F638001009391110092
:1002A00093E111009308D00513850100730000004D
:1002B0000F00F00F930110009308D0051305000004
:1002C00073000000731000C0000000000000000078
:1002D000000000000000000000000000000000001E
:1002E000000000000000000000000000000000000E
:0C02F00000000000000000000000000002
:1010000000000000000000000000000000000000E0
:1010100000000000000000000000000000000000D0
:1010200000000000000000000000000000000000C0
:1010300000000000000000000000000000000000B0
:081040000000000000000000A8
:040000058000000077
:00000001FF
